:2000000002C0178000C004C034C033C032C031C030C02FC02EC02DC02CC02BC02AC029C0D5
:2000200028C027C026C025C024C023C022C021C020C01FC01EC01DC01CC01BC011241FBE59
:20004000CFEFD2E0DEBFCDBF11E0A0E0B1E0E8E7FBE002C005900D92A033B107D9F721E009
:20006000A0E3B1E001C01D92A633B207E1F7B9D181C5C6CF00C000C000C000C000C000C0AD
:2000800000000895D798D698DF98DE980895D79AF1DF1DD00895D69AEDDFD798EBDFD698AE
:2000A000E9DFD79AE7DF13D00895082ED79AE2DF802D0DD0882311F002D0F8CF0895D69A7D
:2000C000D79AD8DFD698D6DFD798D4DF08950894881F01C0880F59F0D69A18F40000D79847
:2000E00002C0D79A00C0C6DFD698C4DFF3CFD69AD798C0DFD698CE9BFECF8827CF9981E0FB
:20010000B9DF99270895882701C081E071E0D69AD798B0DFD698AEDFCE9BFECF8894CF99A5
:200120000894771FA0F7D69A813011F0D79801C0D79AA0DFD698CE9BFECF9CDF872F99271F
:200140000895A0DFE3E6F0E080818064808380818068808386E49BDF87E4B9DFB0DF86E436
:2001600096DF8EE7B4DFABDF86E491DF81E1AFDFA6CFCF92DF92EF92FF9287E488DFC5DFDF
:20018000C82ED12CDC2CCC240D2C000CEE08FF08BADFC82AEE24FF2492DFFF92EF92DF927E
:2001A000CF928EE091E09F938F9351D2C701B60121E730E040E050E0CAD1B901CA0128EE6B
:2001C00033E040E050E09FD19F938F937F936F935F934F933F932F9385E191E09F938F9351
:2001E00036D28DB79EB740960FB6F8949EBF0FBE8DBFFF90EF90DF90CF900895CF93B82FFF
:20020000C62F21E030E0062E01C0220F0A94EAF74AB3422B4ABB40916300522F50954523C2
:20022000409363004BB345234BBB40916000422B4093600088E28A95F1F74AB345234ABB70
:2002400040E44CB944E04DB92F9818B869B945E043BF10BE4FEF5FE088E28A95F1F76599B1
:200260000CC041E049BF12BE48B7416048BFE0E060E070E0CB01AFE014C059B9C9B941506E
:2002800059F7EFCF659B06C0A9B9C9B96F5F7F4F8F4F9F4F08B600FEF5CFF8B7F160F8BF07
:2002A000EF5FEB13F7CF3AB3232B2ABB29B72E7F29BFCF910895A82FB62F21E030E0062E99
:2002C00001C0220F0A94EAF74AB3422B4ABB40916300522F50954523409363004BB34523A0
:2002E0004BBB40916000422B409360004091600041604093600040EC48B988E28A95F1F784
:200300004AB345234ABB40E44CB944E04DB92F9869B945E043BF10BE4FEF88E28A95F1F793
:2003200065990BC041E049BF12BE48B7416048BFE0E060E070E0CB0114C019B8B9B9415090
:2003400061F7F0CF659B06C019B8B9B96F5F7F4F8F4F9F4F08B600FEF5CFF8B7F160F8BFDE
:20036000EF5FEA13F7CF3AB3232B2ABB29B72E7F29BF08951F93CF93DF931F92CDB7DEB7EA
:20038000182F80ED92DE812FA2DE81ED84DEBBDE898395DE89810F90DF91CF911F9108955B
:2003A000CF93DF9380E0E6DFD82F81E0E3DFC82F82E0E0DF1F92DF931F92CF938F731F9219
:2003C0008F9381E291E09F938F9341D18DB79EB708960FB6F8949EBF0FBE8DBFDF91CF91F3
:2003E0000895C298BA9880E091E0909333018093320180916200826080936200A2DE54D0D8
:200400008AE090E037D1CEE0D1E0CADF89E090E031D11BBAD39A61E088E8F0DE9F938F9302
:200420007F936F93DF93CF9312D161E088E843DF9F938F937F936F93DF93CF9308D162E0C7
:2004400088E8DCDE9F938F937F936F93DF93CF93FED062E088E82FDF9F938F937F936F9340
:20046000DF93CF93F4D064E088E8C8DE9F938F937F936F93DF93CF93EAD064E088E81BDFE6
:200480009F938F937F936F93DF93CF93E0D08DB79EB784960FB6F8949EBF0FBE8DBF69DEAF
:2004A0008AE090E0E7D0B1CFE0E0F0E085919491FC01FF733196EE0FFF1FCF018150984195
:2004C0008F3F974030F43697E491EF3F11F0E09374000895BA9A28E62A95F1F798E080FF5E
:2004E00002C0BA9801C0BA9A869528E62A95F1F79150A9F7BA9888E68A95F1F70895EADF55
:2005000080E090E00895A1E21A2EAA1BBB1BFD010DC0AA1FBB1FEE1FFF1FA217B307E40711
:20052000F50720F0A21BB30BE40BF50B661F771F881F991F1A9469F7609570958095909589
:200540009B01AC01BD01CF01089568940013E894A0E0B0E0EDEAF2E01DC0EFEFE7F95901EE
:200560006A015E23550FEE08FE2C87019B01AC019E23990F660B762FCB013BD0CDB7DEB7CB
:20058000EAE024C02F923F924F925F926F927F928F929F92AF92BF92CF92DF92EF92FF926F
:2005A0000F931F93CF93DF93CDB7DEB7CA1BDB0B0FB6F894DEBF0FBECDBF09942A883988D8
:2005C00048885F846E847D848C849B84AA84B984C884DF80EE80FD800C811B81AA81B981B7
:2005E000CE0FD11D0FB6F894DEBF0FBECDBFED010895DF93CF939F92A0E49A2E0024D00118
:20060000E001F00116950795F794E794D794C794B794A79448F41068A20FB31FC41FD51F61
:20062000E61FF71F081E191E220F331F441F551F661F771F881F991F9A9421F79D01AE01DB
:20064000BF01C00111249F90CF91DF910895A0E0B0E0ECE2F3E0A6CFAE014B5F5F4FFA0120
:2006600061917191AF01809132019091330108D0E2E0B4CF6091320170913301DAD108957F
:20068000ACE0B0E0E5E4F3E07DCF7C016B018A01FC0117821682838181FFB0C1CE01019659
:2006A0004C01F7019381F60193FD859193FF81916F01882309F49EC1853239F493FD85919F
:2006C00093FF81916F01853221F4B70190E0B1D1E8CF512C312C20E02032A0F48B3269F003
:2006E00030F4803259F0833269F420612CC08D3239F0803339F4216026C02260246023C044
:20070000286021C027FD27C030ED380F3A3078F426FF06C0852D6AE024D2582E530E13C094
:20072000832D6AE01ED2382E330E20620CC08E3221F426FD5FC1206406C08C3611F4206829
:2007400002C0883641F4F60193FD859193FF81916F018111C1CF982F9F7D9554933028F466
:200760000C5F1F4FFFE3F9830DC0833631F0833771F0833509F057C021C0F80180818983D1
:200780000E5F1F4F44244394512C540114C03801F2E06F0E711CF801A080B18026FF03C052
:2007A000652D70E002C06FEF7FEFC5012C8736D12C0183012C852F77222E16C03801F2E010
:2007C0006F0E711CF801A080B18026FF03C0652D70E002C06FEF7FEFC5012C8714D12C01E2
:2007E0002C852068222E830123FC19C0832D90E048165906A0F4B70180E290E01AD13A9440
:20080000F5CFF50127FC859127FE81915F01B70190E00FD131103A94F1E04F1A510841144F
:20082000510479F7DEC0843611F0893631F5F80127FF07C060817181828193810C5F1F4F0C
:2008400008C060817181072E000C880B990B0E5F1F4F2F76722E97FF09C0909580957095C7
:2008600061957F4F8F4F9F4F2068722E2AE030E0A40117D1A82EA81843C0853729F42F7EFA
:20088000B22E2AE030E025C0F22FF97FBF2E8F36C1F018F4883579F0ADC0803719F088375F
:2008A00021F0A8C02F2F2061B22EB4FE0DC08B2D8460B82E09C024FF0AC09F2F9660B92E9E
:2008C00006C028E030E005C020E130E002C020E132E0F801B7FE07C0608171818281938130
:2008E0000C5F1F4F06C06081718180E090E00E5F1F4FA401D6D0A82EA818FB2DFF777F2EAF
:2009000076FE0BC0372D3E7FA51450F474FE0AC072FC08C0372D3E7E05C0BA2C372D03C016
:20092000BA2C01C0B52C34FF0DC0FE01EA0DF11D8081803311F4397E09C032FF06C0B394B4
:20094000B39404C0832F867809F0B39433FD12C030FF06C05A2CB31418F4530C5B18B32C9B
:20096000B31460F4B70180E290E03C8762D0B3943C85F6CFB31410F43B1801C0312C34FFA1
:2009800011C0B70180E390E03C8753D03C8532FF16C031FD03C088E790E002C088E590E0DE
:2009A000B7010CC0832F867851F031FF02C08BE201C080E237FD8DE2B70190E03AD0A514B2
:2009C00030F4B70180E390E034D05A94F8CFAA94F401EA0DF11D8081B70190E02AD0A110A3
:2009E000F6CF332009F45DCEB70180E290E021D03A94F7CFF7018681978102C08FEF9FEFC3
:200A00002C96E2E1DBCDFC010590615070400110D8F7809590958E0F9F1F0895FC016150F6
:200A2000704001900110D8F7809590958E0F9F1F08950F931F93CF93DF93FB01238121FD7D
:200A400003C08FEF9FEF28C022FF16C046815781248135814217530744F4A081B1819D0112
:200A60002F5F3F4F318320838C93268137812F5F3F4F3783268310C0EB01092F182F008447
:200A8000F185E02D0995892BE1F68E819F8101969F838E83812F902FDF91CF911F910F9122
:200AA0000895FA01AA27283061F1203191F1E8946F936E7F6E5F7F4F8F4F9F4FAF4FB1E0EF
:200AC00040D0B4E03ED0670F781F891F9A1FA11D680F791F8A1F911DA11D6A0F711D811D6F
:200AE000911DA11D22D009F468943F91062E000C3019000C000C3019305D3193CEF6CF0100
:200B00000895462F4770405D4193B3E00FD0C9F7F6CF462F4F70405D4A3318F0495D31FD7A
:200B20004052419302D0A9F7EACFB4E0A6959795879577956795BA95C9F700976105710583
:200B400008959B01AC010A2E06945795479537952795BA95C9F7620F731F841F951FA01D67
:200B60000895002480FD060E660F11F08695D1F7802D0895F894FFCF000000020000000024
:200B80007F0200000000252E386C75090025356C752E252E336C750900252E32583A252E1C
:200BA00032583A252E325800FFFFFFFFFFFFFFFFFFFFFFFFFFFFFFFFFFFFFFFFFFFFFFFFAC
:200BC000FFFFFFFFFFFFFFFFFFFFFFFFFFFFFFFFFFFFFFFFFFFFFFFFFFFFFFFFFFFFFFFF35
:200BE000FFFFFFFFFFFFFFFFFFFFFFFFFFFFFFFFFFFFFFFFFFFFFFFFFFFFFFFFFFFFFFFF15
:200C0000FFFFFFFFFFFFFFFFFFFFFFFFFFFFFFFFFFFFFFFFFFFFFFFFFFFFFFFFFFFFFFFFF4
:200C2000FFFFFFFFFFFFFFFFFFFFFFFFFFFFFFFFFFFFFFFFFFFFFFFFFFFFFFFFFFFFFFFFD4
:20196000FFFFFFFFFFFFFFFFFFFFFFFFFFFFFFFFFFFFFFFFFFFFFFFFFFFF98005FC3FFFFC9
:2019800017C0197A1085931509021200010100803209040000000000000012011001FF009F
:2019A0000008D01653070002000000010403090411241FBECFEFD2E0CDBFDEBF21E0A0E09C
:2019C000B1E001C01D92AC32B207E1F78FC1A82FB92F80E090E041E050EA609530E009C08F
:2019E0002D9182279795879510F084279527305EC8F36F5FA8F30895EADF8D939D930895CC
:201A0000CF93CFB7CF93C395B19BE9F7B19B09C0B19B07C0B19B05C0B19B03C0B19B01C0A3
:201A2000A7C0DF93C0910E01DD27CA5EDE4FB19B02C0DF91EBCF2F930F931F9306B32FEFEF
:201A400001FB20F94F933F9316B34FEF012701FB21F93BE031C04E7F012F16B3216028C03D
:201A6000102F4D7F2260000006B329C04B7F2460012F000016B32BC016B3477F28602AC004
:201A80004F7E06B320612CC04F7D16B320622FC04F7B06B3206432C0422706B349934FEF18
:201AA0000000102711FB20F916B31370C9F1297F91F2012701FB21F906B3237F89F2315004
:201AC00058F1102711FB22F916B3277E79F2012701FB23F92F7C81F206B3102711FB24F90F
:201AE0002F7971F200C016B3012701FB25F92F7359F200C006B3102711FB26F9223040F2C4
:201B000000C016B3012701FB27F9243028F64F77206816B30000F9CF10E21ABF00271DC0D8
:201B20003B503195C31BD04010E21ABF0881033C19F10B3409F120910C011981110F1213F3
:201B4000EDCF093641F10D3211F0013E39F7CAE01AB715FD02C0CA95D9F7009314013F91B3
:201B60004F911F910F912F91DF91CAB7C5FD4BCFCF91CFBFCF91089520911401222379F346
:201B8000109112011123E1F43430E2F03093120120930D0117C00091120101308CF40AE5A0
:201BA00030910F0134FD10C000930F01C1E0D1E00FC02795A8F45150A9F4220F0000F9CF00
:201BC0004AE503C042ED01C0432FC4E1D0E032E017B31360C19A17BB08B320E413E05F933C
:201BE000012756E008BB279520F4515021F4220FF9CF012756E000003B5A08BBD0F2279511
:201C000028F4515029F4220F0000F9CF012756E0279508BB20F4515021F4220FF9CF012729
:201C200056E02991332308BB21F60C7F10911301110FC651D04008BB11F010930C0110E297
:201C40001ABF026017B31C7F402F4C7F5F9100C000C008BB17BB48BB82CF2FEFB0E8A0E01B
:201C60004BE0B093740000008EE599E0B199FECFB19BFECF0197B199FDCFB09B09C096B35B
:201C80009370E9F796B39370D1F7B19BFECFECCF97FF03C0BA1B819501C0BA0FA69541F43B
:201CA000A0E430F4281718F030917400282FA1E04150B9F63093740000000895F20130975A
:201CC00049F02AE7421629E1520631F48091740090E002C08FEB9CEC21E00C01209357000A
:201CE000E8951124CF0102962C01089580917400282EEAE7F9E1E491EF3F19F0E0937400E7
:201D0000000004B601FC06C0EDE7F9E1E491EF3F09F055C114BE88ED8093710087E081BD76
:201D2000B99A2FE78CEF9AE0215080409040E1F700C00000B9988AE580930F018FEF809338
:201D4000000180B5816080BD8BB780628BBFC298712C312C412C512C14E1C0EADFE086B3EC
:201D6000837009F014E1115029F41092130110920C0173DF0AB605FE03C042DE712C03C047
:201D80002197209761F7A895809174002092740022E032120CC0E0E8F9E1E054F10993E03F
:201DA00090935700E8953097C1F7412C512C90E439120AC0F2013297E03829E1F20720F44F
:201DC00095E090935700E8958093740084E0381203C0CD2B11F4EFC0312C8091120183509F
:201DE00087FD98C090910D019D3209F091C0883009F08EC083EC809301018AE580930F01AA
:201E000090911701907680911801992361F1811108C082E899E1909311018093100126E0AE
:201E20006CC0813059F44114510409F44CC080911B01807F482E50901C0145C0833081F4F9
:201E40008091190190911A0139DF80911B0190911C0134DF842D8F70B1F580E4382E33C072
:201E60008F73382E30C09091190110920A01811106C010920B018AE091E022E03AC0853090
:201E800019F49093130127C08630F9F480911A01813019F48AE999E104C0823041F488E882
:201EA00099E1909311018093100122E126C0833051F4911108C08CEA99E1909311018093CC
:201EC000100124E01AC020E018C0883079F0893031F4909315018AE091E020E00AC021E05D
:201EE0008A3009F020E08AE091E003C085E191E021E0909311018093100180911E0181119E
:201F000005C080911D01821708F4282F209300011092120180910F0184FF31C080910001D1
:201F20008F3F69F1C82F893008F0C8E08C1B809300018091010198E8892780930101CC2327
:201F400091F0E0911001F091110182E091E0DC0124912D9331962C2F280F2A13F9CFF093E5
:201F60001101E09310016C2F82E091E045DDCC5FCC3019F08FEF80930001C0930F01C30152
:201F800001963C01803B944029F4EDE7F9E1E491EF3F89F4862D8C7411F0BA9801C0BA9AD8
:201FA0000AB605FED9CE88E1B09988E18150E1F780E28ABFD1CEBA98B99A1BBE10BC2092AD
:081FC00074000000DBCCFFCF30
:00000001FF
